:020000020000FC
:1000000008C018951895189518951895189518956D
:1000100018950FE30EBBE09A0DB301BF0BE107BBD0
:1000200004E008BB1127442706B302FFFDCF06B347
:10003000139500C000C000C000C000C0000002FD59
:10004000F6CF4395443608F002C01127EDCF123D9C
:1000500048F71A3A38F3312F4427C19A3AD039D0A9
:1000600038D037D036D0C19834D033D032D031D018
:1000700030D043954A3F88F31127442706B302FF47
:10008000FDCF06B3139500C000C000C000C000C083
:10009000000002FDF6CF4395443608F002C0112758
:1000A000EDCF123848F7103538F3212F02E0200F3A
:1000B0004427C19A0ED00DD00CD00BD00AD0C198D5
:1000C00008D007D006D005D004D043954A3F88F326
:1000D00001C0089511271EBD532F521B5350052FE9
:1000E0000DBD05E600BF0EE001BD06B302FFFDCF6A
:1000F000A89506B3139500C000C000C000C000C0A2
:1001000002FDF6CF121710F0121B01C011271EBD01
:040110001127EBCFF9
:00000001FF
